:020000002B28AB
:08000800D400030E8301D500B2
:100010008630810004308506D603031D252808306C
:10002000D600D908031DD903A215D703031D1D2827
:100030006430D700DA08031DDA03D803031D25282E
:100040006430D800DB08031DDB030B11550E830061
:10005000D40E540E0900AB0180228316183085009F
:100060000630860024309800413099008312903089
:10007000980007309F00033085000030860008306C
:10008000D6006430D700D8004522A201A215AC22C8
:100090005E08DB00D901DA011030DF08031DDF0044
:1000A000A30185195C280C30AB008022A303031D3B
:1000B00051281F212E232B288316473081008312BD
:1000C00086308100A0308B00A219E9203008AD00F5
:1000D0003208AE003430AF00DB0803199E2105085A
:1000E00010395F0603199828A920A21C7F28E00870
:1000F00003198B28D90803198B28D90186283108C0
:10010000AD003308AE004430AF009E215D08DA0038
:100110006430D700A215DA08031D64288611C820B0
:10012000D901E920050810395F06031D9228A1288E
:10013000221CA128A21CA1280830D6005C08D900E6
:10014000A215B520D908031DA8288611C820DA01F8
:10015000642822180800403019215230A00076226D
:100160005830A000762222140800221C08004030DB
:100170001921E22022100800A21808004C30192191
:100180005430A00076225830A0007622A214080035
:10019000A21C08004C301921E220A21008002219EC
:1001A0000800463019214930A00076224430A000D2
:1001B000762222150800221D080046301921E2206F
:1001C000221108002030A00076222030A0007622E4
:1001D0000800A2115A08052142301921FE203030B2
:1001E000A00076225B08052148301921FE2030301E
:1001F000A0007622590805214E3019212508A000BB
:1002000076222708A00076220800A501A7000A3060
:100210002702031C0E29A700A50A07290A30250278
:10022000031C14290730A5073030A5073030A70775
:10023000080085108038A000762285140800003060
:10024000192104308A000030A50025082E2100382D
:1002500003190800A0007622A50A25298200003093
:10026000080000304A21692911304A2918304A29EA
:100270001F304A292C304A293A304A2943304A292A
:100280004D304A2958304A2962304A296D304A296E
:100290007C304A29A50004308A0025082E21003828
:1002A00003190800A6008321A50A4D2944308400C3
:1002B0005B2934308400000803190800A60083215C
:1002C000840A5B2905212508A60083212708A600AA
:1002D00083210D30A60083210A30A60083298400E3
:1002E0008A212608A700832127080D3C03198129AC
:1002F000271BA71227088000840AA503031D702965
:100300000800800108008316981C8429831226089F
:10031000990008008F2103198A29A60008001808EF
:100320000639031998291A08181218160315080017
:1003300003158C1E08001A0803110800CF20A2180C
:10034000AC298615BC20AB0180228022802280222D
:10035000AC215C08D9000800B421DB205E08DB007A
:100360006430D800A21508002F0884000008031983
:10037000D629A600203C031DC2292422242224229F
:10038000840AB62926082F3C031DD329E830A6008D
:10039000EB21EB21EB21E030A600EB21EB21242225
:1003A0002422840AB629D721840AB62908000430F9
:1003B0008A0041302602031CF729193C031CEA2954
:1003C000193C8A3EF421A600EB21EB21EB21EB2125
:1003D000242224220800A60DA70DA60D270D0339FF
:1003E000A700031D102A08008200003008003030EA
:1003F000A602031C0A2A0A30260203180A2A0A3E09
:10040000A43EF421A6000B220B220B220B220B226E
:10041000242224220800A701A60D0318A70A102AE7
:100420000330271C0130A3002E08A40006142D0859
:10043000302206102D083022A403031D162AA30320
:10044000031D142A242208002E08A40000002D08F1
:10045000302200002D083022A403031D262A0800A4
:10046000AB000000000000000000000000000000E1
:10047000000000000000000000000000000000007C
:100480000000AB03031D312A0800AB018022851058
:100490003030A1006A220530AB0080223030A1004C
:1004A0006A226430AB0090223030A1006A222030F2
:1004B000A1006A222830A00076220130A000762216
:1004C0000230AB0080220630A00076220C30A00063
:1004D0007622080006080F39210486000000051462
:1004E000000005102830AB00902208002008F039E9
:1004F000A1006A2220080F39A100A10E6A2208007B
:10050000E330AC000000000000000000000000002C
:100510000000AC03031D822AAB03031D802A0800E0
:10052000AB03031D902A080083169B001C141A08B5
:100530008312080083169A001C158B1355309D00FA
:10054000AA309D009C148B179C18A42A1C1183129E
:100550000A30AB008022080021309422DD002030D8
:100560009422DC0022309422DE0023309422B0005A
:1005700024309422B20025309422B10026309422F7
:10058000B30027309422DF0028309422E000851049
:100590008030A00076228514A5013430840025081F
:1005A0009422800080040319DA2AA0007622840AAB
:1005B000A50ACF2A1030A5004430840025089422D3
:1005C0008000800403190800840AA50ADE2A21306D
:1005D0002A235D089A2220302A235C089A2222309E
:1005E0002A235E089A2223302A2330089A222430B4
:1005F0002A2332089A2225302A2331089A222630CB
:100600002A2333089A2227302A235F089A22283087
:100610002A2360089A2200302A23343084000008FC
:100620009A220008800403191B2B840A83169B0A54
:1006300083120F2B080010302A2344308400000856
:100640009A220008800403190800840A83169B0A72
:1006500083121F2B83169B008312080069216921D6
:1006600031218A23692134210F30A50034306F21D4
:10067000C30169213E210330A50028306F21B42336
:10068000B000692140210330A50028306F21B42338
:10069000B200692136210F30A50044306F21D3010B
:1006A000692142210330A50028306F21B423B10015
:1006B000692144210330A50028306F21B423B30001
:1006C000692138210330A50028306F21B423DC00D4
:1006D00069213A210330A50028306F21B423DD00C1
:1006E00069213C210330A50028306F21B423DE00AE
:1006F000692146210230A50028306F21B423E00093
:10070000692148210230A50028306F21B423DF0081
:100710006921E72269213421592169213E213008CC
:10072000622140213208622136215621692142216D
:100730003108622144213308622138215C0862219A
:100740003A215D0862213C215E0862214621600851
:10075000AD2348215F08AD2308000038031D013098
:10076000303EA600832169292908031DBB2B2808D8
:10077000A9003030A800A6013030A802A80803194B
:10078000C52B0A30A607A803BE2B3030A902A90842
:0E0790000319CD2BA60AA903C72B26080800C3
:100800005334453454345534503420344D344F34FB
:1008100044344534203420342034203420342034EF
:100820000034433441344C344C3431343A340034A1
:10083000433441344C344C3432343A340034483448
:1008400041344E3447345534503428342E34313406
:10085000533429343A340034543449344D34453413
:100860004F345534543428343134303453342934EB
:100870003A34003449344434283431343034533435
:1008800029343A34003443345734203454344F3408
:100890004E34453431343A34003443345734203400
:1008A0005334503445344534443431343A340034CC
:1008B00043345734203454344F344E344534323476
:1008C0003A340034433457342034533450344534AC
:1008D0004534443432343A3400344D344F344434A3
:1008E0004534283430343D3441342C3431343D34B3
:1008F000423429343A340034533451344C3428349B
:1009000030343D3450342C3431343D344E34293479
:100910003A340034B034EA34EE34E8348034AE345F
:10092000F834AA34A034BF34EC34BA34F034E034B0
:10093000FC34BE34FB34B834A834C034AC34AB34EB
:10094000BC34EB34EF34FA34F834783438341834B7
:0C095000083400348034C034E034F0344B
:02400E00623F0F
:108000004400450020004A005200310057004E0055
:0280100000006E
:108020004400450020004A005200310057004E0035
:0280300000004E
:108040000A0012003C004E001E004E0028000100F5
:0280500001002D
:00000001FF
